:020000020000FC
:1000000005C071C0189582C01895189505E007BB0A
:1000100000E008BB01E003BF02E009BF03E005BF49
:1000200000E40BBF06B301FBEEF306B301FBEEF7F2
:1000300000E60ABF0DE001BD789403D014D0A89566
:10004000FCCF30FB7EF0042D083060F0073250F416
:10005000053110F4497F06C00B3110F0466002C034
:1000600042604B7F0895042F0670002341F400E0A6
:1000700008BB3D7FF89466247724789433C0F894C5
:10008000162D272D789441FB3EF0C0983D7FF894C3
:1000900066247724789421C032600AE1011706E0D3
:1000A000020710F0C09A19C00EE4011702E102071E
:1000B00010F0C09812C008E6011708E1020710F01E
:1000C000C09A0BC009E001170DE3020710F0C098B9
:1000D00004C0F89466247724789442FB16F0C29802
:1000E00001C0C29A08952FB640FB56F0442450E058
:1000F00052BF52E058BF316052E055BF416004C06A
:100100003E7F53E055BF4E7F2FBE18952FB630FB74
:100110000EF4439431FB1EF4639409F473942FBEE0
:02012000189530
:00000001FF
